:020000020000FC
:200000000040003408408C140800683A0000000000000000000000000000000000000000DA
:20000800DEFFED04DFC00015D8400215D8800315D8C00415D9000515D9400615D98007156A
:20001000D9C00815000B307ADA000915DA400A15DA800B15DAC00C15DB000D15DB400E15C4
:20001800DB800F15DBC01015D9401115EBFFFF04DBC012150009313A2880004C10000326FA
:200020002000022600000FC000000706DF401215E8BFFF17E93FFF0400001D001000021E21
:20002800EBFFFF04DBC01215D9401117DF401217DFC000172801707AD8400217D880031714
:20003000D8C00417D9000517D9400617D9800717D9C00817DA000917DA400A17DA800B17F2
:20003800DAC00C17DB000D17DB400E17DB800F17DBC01017DEC01304EF80083ADEFFF90429
:20004000DFC00615DF000515DF0005040001883A0005313AE0BFFE15E0BFFE17E0BFFB15BD
:20004800E03FFD1500800044E0BFFC15E0FFFB17E0BFFC171884703A10001426008000340C
:20005000109CC004E0FFFD17180690FA10C5883A10C0001700800034109CC004E13FFD17AF
:20005800200890FA1105883A10800104108000171009883A183EE83A0001883A0005313A3C
:20006000E0BFFF15E0BFFF1700000706E0BFFC171085883AE0BFFC15E0BFFD1710800044CB
:20006800E0BFFD15003FE106E0BFFB15E0BFFB17103FDB1E0001883A0001883AE037883A9A
:20007000DFC00117DF000017DEC00204F800283ADEFFFB04DFC00415DF000315DF00030454
:20007800E13FFF1500BFFFC4E0BFFD15E03FFE15D0A0181710000726D0A01817E0FFFD1761
:20008000E1BFFE17E17FFF171809883A103EE83A00000206003DA03A0005883AE037883A23
:20008800DFC00117DF000017DEC00204F800283A06C000B4DEC0001406800034D6BC9D1484
:2000900000035840003FFF06DEFFFB04DFC00415DF000315DF000304008000B41084000434
:20009800E0BFFF15E03FFD1500001D0600800104E0BFFE1500001506E0BFFE17113FFFC428
:2000A000008000341095F104E0FFFD1718C7883A18C7883A1907883A18C7883A18C7883A99
:2000A80010C5883A10C00017E0BFFF1710C00015000323C0E0BFFF1710800104E0BFFF153D
:2000B000E0BFFE1710BFFFC4E0BFFE15E0BFFE1700BFE916E0BFFD1710800044E0BFFD158E
:2000B800E0BFFD1710800110103FE01E0007883A008000B41084190410C0003500C00044D0
:2000C000008000B41084180410C00035010000342116010400003DC0003FFF06DEFFF604AE
:2000C800DC0007152021883A2809883ADC400815DFC009152823883A00003F0010C00044D4
:2000D000D88001150080003410960304D880021500800044D880031500800084DC40001569
:2000D800D8C00615DEC00415D88005158000022680800E1710001426814002172880030B85
:2000E00010C8000C1800061E2900191700F7FFC41088001420C6703A2880030D28C01915C3
:2000E800D98004048009883A000083801000091E00800284DFC00917DC400817DC00071718
:2000F000DEC00A04F800283A8009883A00007E80003FE90600BFFFC4003FF6060080003402
:2000F800109C9E04200B883A11000017000031C1208000CC100020262080000710002026D4
:200100002005883A0000020610C00007180018261080004410C000CC183FFB1E10C00017FC
:2001080001FFBFF439FFBFC400CA303A01A0207419C7883A31A020041946703A1986703A17
:200110001800091E1080010410C0001719CB883A00C6303A28C6703A1986703A183FF926E7
:20011800000001061080004410C00007183FFD1E1105C83AF800283A2005883A003FE7061E
:200120000005883AF800283A0005883AF800283A01400034294910040000DC41DEFFF7048D
:2001280000C00034DFC00815DDC00715DD800615DD400515DD000415DCC00315DC80021582
:20013000DC400115DC00001518C124042400011720C00F152080BB0400C000C420C0B915BA
:200138002080BA152000B81505C00204008001042025883AB80D883A81001704000B883A04
:200140008000001580000115800002158080030D800019158000038D8000041580000515DC
:20014800800006150001A1C00580003494400217054000340500003404C00034B5883F04CA
:20015000AD485604A50875049CC88C04858008158540091585000A1584C00B158400071579
:20015800008002848880030D00800044B80D883A89001704000B883A880000158800011572
:2001600088000215880019158880038D8800041588000515880006150001A1C0940003179C
:20016800008004848C4007158D8008158D4009158D000A158CC00B158080030D0080008446
:20017000800000158000011580000215800019158080038D800004158000051580000615A1
:20017800B80D883A000B883A810017040001A1C000800044840007158580081585400915AC
:2001800085000A1584C00B1590800E15DFC00817DDC00717DD800617DD400517DD00041700
:20018800DCC00317DC800217DC400117DC000017DEC00904F800283A0005883AF800283ADF
:20019000DEFFFC04DC8002152825883ADC00001501401A042021883A913FFFC4DFC0031553
:20019800DC400115000310008009883A11401D041023883A0000E8801021883A10000726B8
:2001A0001100030410000015148001151100021589801A04000B883A0001A1C08005883A93
:2001A800DFC00317DC800217DC400117DC000017DEC00404F800283ADEFFFB04DC00001515
:2001B00004000034841C9D04DCC003152027883A81000017DFC00415DC80021520800E1771
:2001B800DC4001151000021E000049C0810000172480B804047FFFC4910001179400021728
:2001C000213FFFC420000A168080030F10000C2680C01D040000020618BFE60F10000826F5
:2001C800213FFFC41C3FFD0418C01A04247FFA1E9080001710001D261025883A003FEE0643
:2001D00000BFFFC48080038D008000448080030D80001915800000158000021580000115B9
:2001D80080000415800005158000061501800204000B883A810017040001A1C08005883AA0
:2001E00080000C1580000D158000111580001215DFC00417DCC00317DC800217DC40011756
:2001E800DC000017DEC00504F800283A014001049809883A0000640090800015103FDE1E86
:2001F00000800304988000150005883A003FF00600800034109C9D041100001701400034A1
:2001F800294910040000DC4120800E1710000126F800283A000049C1F800283AF800283A30
:20020000F800283AF800283A00800034109C9E04110000170140003429418E040000D001BE
:2002080000800034109C9E041100001701400034294122040000D001308002171000672670
:2002100028C0030BDEFFF404DD400715DD000615DC000215DFC00B15DF000A15DDC0091567
:20021800DD800815DCC00515DC800415DC4003151880020C2821883A202B883A3029883A14
:200220001000272628800417100025261880008CA440001710002A2605A000340027883A02
:200228000025883AB5BF0004980D883AA809883A90004626900F883AB480022E01E00034A7
:2002300039FF00048080091781400717103EE83A00805A0EA0C0021798A7883A90A5C83A6A
:200238001885C83AA0800215103FEF1E0005883ADFC00B17DF000A17DDC00917DD800817B3
:20024000DD400717DD000617DCC00517DC800417DC400317DC000217DEC00C04F800283A07
:20024800800B883AA809883A000229801000EE1E80C0030BA44000171880008C103FD61E5F
:200250001880004C1000421E0039883A0025883A90001A261880800C84C0021710002126B0
:20025800982F883A94C096361881200C1000A11E81000017B80D883AE00B883A00018C00F0
:2002600080C00217810000179005883A1CE7C83A25CF883A84C0021581C00015A0C0021751
:20026800E0B9883A90A5C83A18A7C83AA4C00215983FCE2680C0030B903FE61E8F00001716
:200270008C8001178C400204003FE1068CC000178C8001178C400204003FB3060005883A3A
:20027800F800283A810000178080041711005A3685C0051795C0583600A0003410BFFFC40E
:200280009009883A1480012E1009883AB80B883A0002F4C0B80B883A1009883A00031000B7
:200288008140071780C00917100F883AE00D883AA809883A183EE83A00BFD8168080030BE1
:20029000108010148080030D00BFFFC4003FA8060027883A0011883A0039883A0025883A7D
:2002980090001F2640005A26982D883A94C0012E902D883A8100001780800417B02F883AD4
:2002A00081C005171100032E80C0021738C7883A1D801816B1C03E168080091781400717F6
:2002A800E00D883ADA000115A809883A103EE83A102F883ADA00011700BFE00E9DE7C83A8E
:2002B00098001F26A0800217E5F9883A95E5C83A15EFC83AA5C00215B83F8426903FE11E0B
:2002B8008F0000178C8001170011883A8C400204003FDB06180D883AE00B883ADA00011513
:2002C000D8C0001500018C00D8C0001780800017800B883AA809883A10C5883A80800015B2
:2002C800D8C0001500027600D8C00017DA000117103FC21E182F883A9DE7C83A983FE11EBC
:2002D000800B883AA809883A00027600103FBB1E0011883A003FDB0694C0012E9027883ABF
:2002D800980D883AE00B883A00018C008080021780C0001714C5C83A1CC7883A808002155E
:2002E00080C00015100043269805883A003F8306B00D883AE00B883ADA00011500018C0060
:2002E8008080021780C00017DA0001171585C83A1DAD883A8080021585800015003FBF0637
:2002F000810000179027883A902F883A003F6906900D883A01400284E009883A0001694033
:2002F80010003E26108000441727C83A02000044003F9D06808005178140041781C00017E6
:2003000010A7883A9885883A1026D7FA396DC83AB10000449885883A1027D07A2485883A16
:20030800980D883A9880022E1027883A100D883A18C1000C18001C26300B883AA809883A9F
:200310000000E880102F883A1000292681400417B00D883A1009883A000177808080030BC9
:2003180000FEDFC410C4703A108020148080030DBD89883A9D8FC83A85C0041584C00515E0
:20032000810000159027883A81C00215902F883A003F3806800B883AA809883A0002760020
:20032800103FB926003F6506A809883A0001B440102F883A103FEE1E81400417A809883ACA
:20033000000291008080030B00FFDFC41884703A00C00304A8C00015003F590694C00044AA
:2003380002000044003F600600BFFFC4003F000600800304A88000158080030B003F50068C
:20034000DEFFF704DD000415DFC00815DDC00715DD800615DD400515DCC00315DC80021584
:20034800DC400115DC0000152500B804A0002326282B883A002F883A0580004404FFFFC413
:20035000A4400117A48002178C7FFFC488000D1694000304948003848080000B8C7FFFC4CC
:20035800813FFD04B080042E9080000F14C00226A83EE83AB8AEB03A84001A0494801A041B
:200360008CFFF51EA5000017A03FED1EB805883ADFC00817DDC00717DD800617DD4005178E
:20036800DD000417DCC00317DC800217DC400117DC000017DEC00904F800283A002F883A35
:20037000003FF206DEFFF704DD000415DFC00815DDC00715DD800615DD400515DCC0031590
:20037800DC800215DC400115DC0000152500B804A0002326282B883A2027883A002F883AF6
:200380000580004404BFFFC4A4400117A40002178C7FFFC488000C16840003048080000B47
:200388008C7FFFC4817FFD04B080052E8080008F9809883A14800226A83EE83AB8AEB03A1D
:2003900084001A048CBFF51EA5000017A03FEE1EB805883ADFC00817DDC00717DD80061734
:20039800DD400517DD000417DCC00317DC800217DC400117DC000017DEC00904F800283ABD
:2003A000002F883A003FF206DEFFF504DC800315DFC00A15DF000915DDC00815DD800715DD
:2003A800DD400615DD000515DCC00415DC400215DC000115288002C400C005842025883A6E
:2003B00018807F2E047FFE041462703A8800A3168940A2360003600000807DC41441E92ED1
:2003B8008804D27A1000A12600C0010418811E368804D1BA12000E4411C00E044209883A59
:2003C00004C000342109883A9CD719042109883A9909883A24000117213FFE0424009726DA
:2003C8008080011701BFFF04014003C41184703A1447C83A28C007161800920E840003173B
:2003D00024008E26808001171184703A1447C83A28FFF90E3809883A018000349C000417E4
:2003D80031971904320002048201342680C0011700BFFF04188E703A3C45C83A00C003C497
:2003E00018811F16320005153200041510007F0E00807FC411C0FD363806D0FA01C0004427
:2003E8003080011719400044294B883A1807D0BA294B883A294B883A298B883A38C6983AFF
:2003F00029C000172A7FFE041886B03A8240031581C0021530C001152C0000153C000315ED
:2003F8002005D0BA01400044288A983A19406F3628C4703A10000A1E00BFFF04294B883A69
:200400002088703A28C4703A210001041000041E294B883A28C4703A21000104103FFC2639
:2004080002BFFF04024003C421800044318D883A318D883A318D883A998D883A333FFE0446
:200410002017883A318001043400001731FFFD0481C0041E0000FB061801030E8400031775
:2004180081C0F826808001171284703A1447C83A48FFF90E80800317810002178940005491
:200420008140011520800315110002158463883A9C4005159C400415188000548880011567
:200428008A0003158A00021588E3883A88C000159009883A000362408080020400001B06C0
:20043000044004048940253600036000008001840100008404C000341085883A9CD7190470
:200438001085883A9885883A1400011710FFFE0480C0D92680C001178100031700BFFF043D
:200440001884703A814002178085883A10C00117290003152140021518C0005410C0011502
:200448009009883A0003624080800204DFC00A17DF000917DDC00817DD800717DD4006175E
:20045000DD000517DCC00417DC800317DC400217DC000117DEC00B04F800283A00800304AF
:20045800908000150005883A003FF006010020040200100401C00FC4003F61064009883AE3
:20046000003F750681000317003FDE0681C5883A114001179009883A294000541140011514
:200468000003624080800204003FE0069C00021700BFFF0485800117B0AC703AB4400336DD
:20047000B445C83A00C003C418805D1605C0003400800034109CAD04BDDC9F04154000172D
:20047800B8C0001700BFFFC4858D883A8D6B883A1880EA26AD4403C400BC0004A8AA703AA9
:20048000A80B883A9009883AD980001500020A801029883A00BFFFC4D9800017A080E82677
:20048800A180A63607000034E71CB604E0800017A887883AE0C000153500E626B900001731
:2004900000BFFFC42080EE26A185C83A10C5883AE0800015A0C001CC1800BC26A0E9C83A30
:2004980000840204A500020410C7C83AA545883A1083FFCC18ABC83AA80B883A9009883A97
:2004A00000020A8000FFFFC410C0E1261505C83A1545883A10800054E0C000179D00021590
:2004A800A0800115A8C7883AE0C0001584C00E26018003C43580A72E81400117013FFE04B3
:2004B000B0BFFD041104703A2900004C2088B03A81000115014001448089883A2140011597
:2004B800214002153080CD3600800034109CAC041100001720C0012E10C000150080003419
:2004C000109CAB04110000179C00021720C0012E10C0001580C0011700BFFF041886703A8E
:2004C8001C45C83A1C40023600C003C4188004169009883A000362400005883A003F7B065D
:2004D00088C0005480C001158463883A108000549C400215888001159009883A000362407C
:2004D80080800204003F710600C0050418804A2E00C0150418806E368804D33A12001BC4D0
:2004E00011C01B844209883A003EDD063804D27A00C001041880442E00C0050418808136EF
:2004E8001140170410C016C4294B883A294B883A294B883A994B883A288000170180003422
:2004F000297FFE04319719042880652601BFFF0410C001171986703A38C0022E1080021765
:2004F80028BFFB1E1140031798C0011781400315808002152C00021514000315003EF8066E
:2005000088C0005480C001158463883A344005153440041510C000548A0003158A000215BE
:2005080088C0011588A3883A888000159009883A0003624080800204003F3C0630C00117DC
:20051000003EE7065AC00044588000CC31800204103EFD1E0000240614000317143F251E90
:2005180021000084003EBC068085883A10C00117810003178140021718C0005410C00115E8
:2005200029000315214002159009883A0003624080800204003F25061200170411C016C4BA
:200528004209883A003E96063804D1BA11400E4410C00E04294B883A003FBC0684FF592647
:2005300000800034109719041400021700BFFF0480C001171886703A003F910660800217D5
:20053800213FFFC41300651E208000CC633FFE04103FFA1E988001170146303A1884703A4C
:2005400098800115294B883A117F2836283F27262886703A5809883A183EC31E294B883AAD
:200548002886703A21000104183FFC26003EBE0600C05504188012368804D3FA12001E0414
:2005500011C01DC44209883A003E6D0600C40004003F460600800044A0800115003F740615
:200558001805D0BA01C0004430C00117388E983A2805883A38C6B03A30C00115003F9B067A
:2005600000C1550418801A368804D4BA12001F4411C01F044209883A003E5906AD40040457
:20056800003F170600C01504188023363804D33A11401BC410C01B84294B883A003F7B066F
:200570009C00021700BFFF0480C001171886703A003F53063083FFCC103F181E9900021707
:20057800B545883A1080005420800115003F3E0601003F8402001FC401C01F84003E4006F9
:2005800000800034109C9F0415000015003F110600800044002B883A003F1F0681400204FC
:200588009009883A0002910000800034109CB60410C00017003F2C0600C055041880053607
:200590003804D3FA11401E0410C01DC4294B883A003F560600C15504188005363804D4BA96
:2005980011401F4410C01F04294B883A003F4F0601403F8400C01F84003F4C0698800117AA
:2005A000003FA0068808D0FA208000441085883A003E9006208000CC280F883A100034261E
:2005A80030BFFFC430001A2620C0000329803FCC30C0051E000018061000152620C000031B
:2005B00010BFFFC430C014262100004420C000CC183FF91E020000C44080113610000C26E1
:2005B80020C0000329403FCC28C00B2620C0004439803FCC2089883A0000030618C000443B
:2005C000197FFFC3314005261805883A20FFFB1E0005883AF800283A2005883AF800283AAC
:2005C80028C03FCC1812923A02FFBFF402A0207448D2B03A4806943A5AFFBFC452A020042E
:2005D00048D2B03A20C0001748C6F03A1ACD883A00C6303A30C6703A1A86703A183FE01EC0
:2005D80010BFFF042100010440BFF636003FDB063005883A003FD706DEFFFD04DFC0021519
:2005E000DC400115DC00001500C003C42005883A1980452E2906B03A18C000CC1800441E27
:2005E800347FFC048822D13A28C00104234001048820913A2B00020422C00204840005041D
:2005F0002A800304224003042C21883A2811883A200F883A410000171FC0001763C000174E
:2005F80039000015538000176FC000155BC000154B80001518C0040439C00404420004042C
:200600006B400404630004045AC00404528004044A4004041C3FEF1E89C00044380E913A28
:20060800310003CC02C000C411C7883A29CB883A5900212E1813883A2811883A200F883A7B
:20061000428000174A40010439FFFF044ABFFF154200010459FFFA36213FFF042008D0BA26
:20061800318000CC210000442109883A2109883A1907883A290B883A30000626198D883A6C
:2006200029C0000318C000442940004419FFFFC519BFFB1EDFC00217DC400117DC00001759
:20062800DEC00304F800283A2007883A003FF2062007883A003FF106200D883A003FEE0652
:200630002005883A29000B2E298F883A21C0092E2187883A198BC83A3000482639FFFFC426
:200638003900000318FFFFC41900000528FFFB1EF800283A00C003C41980412E2886B03AAD
:2006400018C000CC1800401E33FFFC04781ED13A28C0010413400104781C913A2B000204D8
:2006480012C00204738005042A800304124003042B9D883A2811883A100F883A41000017F6
:2006500039C0040418C00404393FFC15193FFC176B4004045AC00404693FFC1561000017AF
:200658004A40040442000404593FFC15510000176300040452800404493FFC151BBFEF1ED0
:20066000790000442008913A328003CC02C000C41107883A290B883A5A801E2E1813883AE0
:200668002811883A500F883A410000174A40010439FFFF04493FFF154200010459FFFA36C9
:20067000513FFF042008D0BA318000CC210000442109883A2109883A1907883A290B883A93
:2006780030000B26198D883A29C0000318C000442940004419FFFFC519BFFB1EF800283ABD
:200680001007883A003FF6061007883A003FF506F800283A500D883A003FF10620C000CCD8
:200688002005883A1800442631FFFFC4300040262813883A200D883A2007883A0000040681
:200690003A3FFFC43180004438003926400F883A18C00044324000051A0000CC403FF81E63
:20069800010000C421C02D2E29003FCC200C923A3108B03A200C943A218CB03A010003C499
:2006A00021C0182E3B3FFC046018D13A1A0001041AC002046008913A1A8003041813883A56
:2006A800210005041909883A49800015418000155980001551800015420004044A400404C0
:2006B0005AC0040452800404413FF71E630000446018913A39C003CC010000C41B07883A3E
:2006B80021C00E2E1813883A3811883A010000C449800015423FFF044A400104223FFC36C4
:2006C000393FFF042008D0BA39C000CC210000442109883A2109883A1907883A38000526A6
:2006C80019CF883A1940000518C0004438FFFD1EF800283AF800283A2007883A300F883AFE
:2006D000003FC706DEFFF604DC800215DFC00915DF000815DDC00715DD800615DD40051593
:2006D800DD000415DCC00315DC400115DC0000153025883A2800B726282B883A2029883AF9
:2006E00000036000A8BFFF17043FFF0490C002C401000584ACFFFE041420703A20C0332E68
:2006E800047FFE041C62703A8807883A880058168C80573680C0300E07000034E717190491
:2006F000E1C002179C09883A2200011721C06326017FFF84414A703A214B883A29800117FE
:2006F8003180004C30003F261080004C10008326900B883AA009883A0000E8801025883A94
:2007000010011E26A93FFF1710FFFE0400BFFF842084703A9885883A1880EE2681BFFF0417
:20070800008009041180B83600C004C4198096369005883AA807883A1900001711000015BA
:20071000190001171100011518C0021710C00215A80B883AA009883A00029100A009883ABB
:20071800000362409005883A0000120600C004041823883A003FCE06A825883A8445C83A7B
:2007200000C003C418802636998001179C07883A3180004C3420B03A9C000115188001170B
:200728001080005418800115A009883A000362409005883ADFC00917DF000817DDC0071740
:20073000DD800617DD400517DD000417DCC00317DC800217DC400117DC000017DEC00A0400
:20073800F800283A017FFF04414A703A814D883A30C01F162080031720C00217A825883A98
:200740003021883A1880031510C00215003FDB0600800304A08000150005883A003FE50622
:2007480098C001179C4B883A1100005418C0004C1C62B03A9C400115290001152885883AE7
:2007500010C0011729400204A009883A18C0005410C0011500029100003FD306017FFF0487
:20075800414A703A898004048151883A4180590E1080004C103F9E1EADBFFE1700BFFF0455
:200760009DADC83AB18001173084703A2000202680AF883AB96F883A21C05F26B8C01C1635
:200768002080031720C0021781BFFF04010009041880031510C00215B0C00217B080031703
:20077000B48002041880031510C0021521801B36008004C41180352EA8800017B0800215E4
:20077800A8800117B0800315008006C411807F36B0800404AD40020400002D06ADBFFE176A
:2007800000BFFF049DADC83AB10001172084703AB03F772680AF883AB8FF7516B08003172B
:20078800B0C0021781BFFF04010009041880031510C00215B480020421BFE52EA80B883A3E
:200790009009883A00018C00B821883AB027883A003F8A06300B883ADFC00917DF000817A4
:20079800DDC00717DD800617DD400517DD000417DCC00317DC800217DC400117DC00001789
:2007A000DEC00A040000E881A8C0001790C00015A8C0011790C0011500C006C419804536BC
:2007A80090800204A8C00204003F63069005883AA8C00017B821883AB027883A10C0001516
:2007B000A8C0011710C00115A8C0021710C00215003F6A069C67883A4445C83AE4C00215A1
:2007B8001080005498800115A8BFFF17A009883A1080004C1462B03AAC7FFF150003624007
:2007C000A805883A003F6B06A80B883A9009883A00018C00003F4E0689000404B93FBC16AF
:2007C800B0800317B0C0021781BFFF04010009041880031510C00215B48002042180433602
:2007D000008004C411803F2EA8800017B0800215A8800117B0800315008006C411803F3665
:2007D800B0800404AD400204A8C0001710C00015A8C0011710C00115A8C0021710C00215A4
:2007E000B447883ABC45C83AE0C002151080005418800115B0800117A009883A1080004C61
:2007E8001462B03AB4400115000362409005883A003F4006A8C0021790C00215A8C003179C
:2007F00090C003153080112690800404A8C00404003F190690FFFF1700BFFF04A825883ABE
:2007F8001884703A80A1883A003F2406A8800217B0800415A8800317B080051531000A26D8
:20080000B0800604AD400404003FA906A900041790800604A8C0060491000415A9000517FC
:2008080091000515003F0406A8C00417AD400604B0800804B0C00615A8FFFF17B0C0071552
:20081000003F9B069005883A003FC706A80B883A9009883A00018C00003FC906A8800217D9
:20081800B0800415A8800317B080051531000726B0800604AD400404003FBB06A009883AF3
:20082000000362400005883A003F0A06A8C00417AD400604B0800804B0C00615A8FFFF17FF
:20082800B0C00715003FB006DEFFFD04DC00001504000034DC400115841CAE042023883A9F
:200830002809883ADFC0021580000015000380C000FFFFC410C00526DFC00217DC4001177E
:20083800DC000017DEC00304F800283A80C00017183FF92688C00015003FF706DEFFFE0469
:20084000DC0000152821883A2940038FDFC001150002E3C01000071680C014171887883A4E
:2008480080C01415DFC00117DC000017DEC00204F800283A80C0030B18FBFFCC80C0030D03
:20085000DFC00117DC000017DEC00204F800283A0005883AF800283A2880030BDEFFFB042D
:20085800DCC00315DC800215DC400115DC000015DFC0041510C0400C2821883A2023883A52
:200860003025883A3827883A180005262940038F01C00084000D883A0002C2008080030B1C
:200868008140038F10BBFFCC980F883A900D883A8809883A8080030DDFC00417DCC00317EC
:20087000DC800217DC400117DC000017DEC0050400022381DEFFFE04DC0000152821883AA4
:200878002940038FDFC001150002C20000FFFFC410C0082680C0030B8080141518C40014C5
:2008800080C0030DDFC00117DC000017DEC00204F800283A80C0030B18FBFFCC80C0030DE4
:20088800DFC00117DC000017DEC00204F800283A2940038F00023EC1DEFFFD042805883ADF
:20089000DC00001504000034DC400115300B883A841CAE042023883A380D883A1009883AB7
:20089800DFC002158000001500038F8000FFFFC410C00526DFC00217DC400117DC00001747
:2008A000DEC00304F800283A80C00017183FF92688C00015003FF70600800034DEFFFD0441
:2008A800109C9E04DC4001152023883A11000017DC000015DFC002152821883A2000022689
:2008B00020800E17100031268080030B10C0020C1009883A18000F2680C00417180015263A
:2008B8001100004C20001C1E1080008C1000291E808005178080021518001C260005883AA2
:2008C000DFC00217DC400117DC000017DEC00304F800283A2080040C10002E262080010C79
:2008C80010001E1E80C00417208002148080030D183FEB1E1100A00C01408004217FE82613
:2008D000800B883A8809883A0002C8008080030B80C00417003FE20680800517800002155B
:2008D8000085C83A80800615183FE41E80C0030B0005883A1900200C203FE12618C0101449
:2008E00080C0030D00BFFFC4003FDD0600007E80003FCD060005883A003FD60681400C172E
:2008E8002800062680801004288003268809883A000291008100030B80000C1580C0041746
:2008F00000BFF6C41108703A8000011580C00015003FD50600800244888000152080101400
:2008F8008080030D00BFFFC4003FC506DEFFFD04DC00001504000034DC400115841CAE04B9
:200900002023883A2809883ADFC00215800000150003164000FFFFC410C00526DFC00217C6
:20090800DC400117DC000017DEC00304F800283A80C00017183FF92688C00015003FF70643
:2009100028003926DEFFFC04DC400115DC000015DFC00315DC8002152023883A2821883A06
:200918002000022620800E17100027268080030F1000071E0005883ADFC00317DC80021719
:20092000DC400117DC000017DEC00404F800283A800B883A8809883A000254401025883A63
:2009280080800B1710000426814007178809883A103EE83A100016168080030B1080200CAB
:200930001000151E81400C172800052680801004288002268809883A0002910080000C15C2
:2009380081401117280003268809883A000291008000111500007F808000030D00007FC00B
:200940009005883A003FDC0600007E80003FD70604BFFFC4003FE806814004178809883A23
:2009480000029100003FE7060005883AF800283A00800034109C9E04200B883A1100001798
:20095000000244012880030BDEFFFB04DCC00315DC400115DFC00415DC800215DC000015AC
:2009580010C0020C2823883A2027883A1800311E28C00117108200142880030D00C04B0EAD
:200960008A000A17400023269C00001710C4000C98000015180048268980141710C0010C6C
:200968001800062688C0011788800C1730CDC83A1000022688800F17308DC83A8940071795
:20097000000F883A9809883A403EE83A00FFFFC410C0442688C0030B8900041788000115FF
:20097800197DFFCC8940030D8900001518C4000C18002C1E89400C179C000015280005264D
:2009800088801004288002269809883A0002910088000C150005883ADFC00417DCC0031795
:20098800DC800217DC400117DC000017DEC00504F800283A2C800417903FF6262C000017BD
:20099000108000CC2C80001584A1C83A1000131E288005178880021504000316003FED0690
:2009980090A5883A043FEB0E8880091789400717800F883A900D883A9809883A103EE83A7A
:2009A00080A1C83A00BFF61688C0030B00BFFFC418C0101488C0030D003FDF060005883A32
:2009A800003FEC0688801415003FD20628C00F1700FFB316003FD70689400717000D883A0E
:2009B00001C000449809883A403EE83A100D883A00BFFFC4308014268880030B8A000A1713
:2009B800003FAE0698C00017183FBA260100074419000626010005841900042688C0030BD2
:2009C00018C0101488C0030D003FC3068880030B88C004178800011510BDFFCC8880030DF4
:2009C80088C00015003FB30698800017103FEA2600C0074410C0022600C0058410C0031EEF
:2009D0009C0000150005883A003FB30688C0030B3005883A18C0101488C0030D003FAE0603
:2009D800DEFFFD04DC000115DFC002152021883A2000022620800E1710000C262880030F6D
:2009E0001000051E0005883ADFC00217DC000117DEC00304F800283A8009883ADFC002174F
:2009E800DC000117DEC0030400025441D940001500007E80D9400017003FF00620000526E3
:2009F00000800034109C9E04200B883A110000170002760100800034109C9D04110000172E
:2009F800014000342949D8040000DC41DEFFFB04DCC0031504C00034DC800215DC400115D2
:200A0000DC000015DFC004152821883A9CD719042025883A0003600098800217144001178B
:200A080000BFFF0488A2703A8C21C83A8403FBC48020D33A0083FFC4843FFFC48020933A5D
:200A10001400060E000B883A9009883A00020A8098C002171C47883A10C00A269009883AF9
:200A1800000362400005883ADFC00417DCC00317DC800217DC400117DC000017DEC005049F
:200A2000F800283A040BC83A9009883A00020A8000FFFFC410C00D2600C0003418DCB604FD
:200A280018800017990002178C23C83A8C4000541421C83A244001159009883A1C0000153F
:200A30000003624000800044003FE706000B883A9009883A00020A8099000217014003C4A3
:200A38001107C83A28FFDD0E01400034295C9F042940001718C0005420C0011500C000343F
:200A40001145C83A18DCB60418800015003FD30628004126DEFFFD04DC400115DC0000153B
:200A48002023883A2821883ADFC002150003600081FFFF1700BFFF840100003481BFFE0416
:200A50003884703A21171904308B883A2A4001172200021700FFFF0448C6703A2A00572630
:200A580028C0011539C0004C3800091E823FFE1722400204320DC83A31C002171205883A7A
:200A60003A406526320003173A00031541C0021528CF883A39C0011739C0004C38003A2614
:200A680010C0005430C001153087883A1880001500C07FC4188019361004D0FA01C0004451
:200A70002140011710C0004418C7883A1005D0BA18C7883A18C7883A1907883A3884983AE7
:200A780019C000171A3FFE041144B03A3200031531C002152080011519800015398003154D
:200A80008809883ADFC00217DC400117DC000017DEC0030400036241F800283A100AD27A19
:200A880000C0010419404A36100AD1BA28C00E4418C7883A29400E0418C7883A18C7883A73
:200A90001909883A20C0001701C00034213FFE0439D7190420C0442601FFFF041940011729
:200A980029CA703A1140022E18C0021720FFFB1E190003173100031530C0021521800215BC
:200AA00019800315003FDE0629C0021710C5883A00C0003418D71B0438C03B262A0003172A
:200AA800114000543087883A3A00031541C002153140011518800015003FBD0639C0004C2B
:200AB00010C5883A3800071E81FFFE1731CDC83A30C003173140021711C5883A28C0031571
:200AB8001940021510C0005430C0011500C0003418DCA00418C000172180021510FFC0364C
:200AC00000800034109CAD04114000178809883A00027EC0003FBA0628C9883A210001171F
:200AC8002100004C2000391E29C00217290003171885883A10C000543900031521C0021519
:200AD00030C00115308D883A30800015003FAC0600C005041940153628C0170418C7883ABA
:200AD800294016C4003FB406280BD0BA00C0004438800117194A983A2007883A2884B03A7D
:200AE00038800115003FBB06218005152180041510C0005431C0031531C0021530C0011578
:200AE800308D883A30800015003F950600C0150419400536100AD33A28C01BC418C7883AD4
:200AF00029401B84003F9C0600C0550419400536100AD3FA28C01E0418C7883A29401DC474
:200AF800003F950600C1550419400536100AD4BA28C01F4418C7883A29401F04003F8E0663
:200B000000C03F8401401F84003F8B0610C0005430C00115308D883A30800015003F780673
:200B0800DEFFFD042805883ADC00001504000034DC400115300B883A841CAE042023883A51
:200B1000380D883A1009883ADFC002158000001500034A8000FFFFC410C00526DFC0021756
:200B1800DC400117DC000017DEC00304F800283A80C00017183FF92688C00015003FF70631
:200B20002880030B10C0008C1800411EDEFFEC04DC000F152821883A2940038FDC40101518
:200B2800DFC01315DCC01215DC8011152023883A28001C16D80D883A0002E9C010001816B2
:200B3000D880011700E0001410BC000C14C8002010C0372680C0030B18C2001480C0030DB4
:200B380000C8000410C0521E8140038F8809883A0002EF8010004C268080030B80C010C4D6
:200B400080C00015108000548080030D0080004480C004158080051504810004000007067F
:200B48008080030B10C0200C18001F1E04810004108200148080030D0027883A900B883AA9
:200B50008809883A0000E88010002C2680C0030B010000342101240489000F1518C02014E2
:200B580080C0030D80800015808004158480051598001A1EDFC01317DCC01217DC801117FF
:200B6000DC401017DC000F17DEC01404F800283A288010C428800015288004150080004462
:200B680028800515F800283A04801004003FE00681000A1700C0003418C8750420FFC51EA3
:200B70008080030B04810004848013151484B03A8080030D0027883A003FD8068140038FB7
:200B78008809883A0002EF80103FE2268080030B108000548080030D003FDE068080030B0F
:200B800010C0800C183FDB1E1080009480C010C48080030D0080004480C0001580C00415EF
:200B880080800515003FD30604810004003FC3060027883A04810004003FC006DEFFFD0435
:200B90002805883ADC00001504000034DC400115300B883A841CAE042023883A380D883AA0
:200B98001009883ADFC00215800000150003684000FFFFC410C00526DFC00217DC400117C3
:200BA000DC000017DEC00304F800283A80C00017183FF92688C00015003FF706DEFFFD04FF
:200BA8002805883ADC00001504000034DC400115841CAE042023883A300B883A1009883AB4
:200BB000DFC002158000001500032CC000FFFFC410C00526DFC00217DC400117DC0000174F
:200BB800DEC00304F800283A80C00017183FF92688C00015003FF706DEFFFD04DC000015E9
:200BC00004000034DC400115841CAE042023883A2809883ADFC002158000001500033C00D7
:200BC80000FFFFC410C00526DFC00217DC400117DC000017DEC00304F800283A80C000171B
:200BD000183FF92688C00015003FF70620001B16000F883A28001616200D883A29001A2E20
:200BD8000080080400C000440000010610000D26294B883A10BFFFC418C7883A293FFB3621
:200BE0000005883A180007260005883A31400236314DC83A10C4B03A1806D07A280AD07A57
:200BE800183FFA1E380001260085C83AF800283A014BC83A39C0005C003FE7060109C83A63
:200BF00001C00044003FE30600C00044003FEE0620001716000F883A2005883A280012162C
:200BF8002900162E0180080400C000440000010630000A26294B883A31BFFFC418C7883AEE
:200C0000293FFB36180005261806D07A114001361145C83A280AD07A183FFB1E3800012665
:200C08000085C83AF800283A014BC83A003FEC060109C83A01C00044003FE70600C000442B
:200C1000003FF106200D883A2900152E280014160080080400C000440000020610000E2605
:200C180028000516294B883A10BFFFC418C7883A293FFA36180008260005883A31400236C2
:200C2000314DC83A10C4B03A1806D07A280AD07A183FFA1EF800283A0005883AF800283AA8
:200C280000C00044003FF4062005883A2900122E280011160180080400C000440000020637
:200C300030000C2628000516294B883A31BFFFC418C7883A293FFA36180006261806D07A31
:200C3800114001361145C83A280AD07A183FFB1EF800283AF800283A00C00044003FF706DC
:200C40000005883A2000072620C0004C2008D07A180001261145883A294B883A203FFA1EDE
:200C4800F800283AF800283ADEFFFE04DFC00115DF000015D839883AD0A0091710000326B4
:200C5000D0A00917103EE83A00000106D0A01104E037883ADFC00117DF000017DEC00204CE
:200C5800F800283ADEFFFB04DFC00415DF000315DF000304E13FFF15E0BFFF17100008169A
:200C600001400304E13FFF17000310001007883A00800034109825041885883A000001061F
:200C68000005883AE0BFFD15E0BFFD1710001926E0BFFD17108000171080041710000626B1
:200C7000E0BFFD171080001710800417E13FFD17103EE83A000001060005883AE0BFFE153B
:200C7800E13FFF1700037880E0BFFE171000070E000312801007883AE0BFFE170085C83AA9
:200C80001880001500BFFFC4000007060005883A00000506000312801007883A0080144400
:200C88001880001500BFFFC4E037883ADFC00117DF000017DEC00204F800283ADEFFFD04BB
:200C9000DF000215DF000204E13FFE15E17FFF150001883AE037883ADF000017DEC001048D
:200C9800F800283ADEFFFC04DF000315DF000304E13FFD15E17FFE15E1BFFF15E0BFFF171A
:200CA000E037883ADF000017DEC00104F800283ADEFFFE04DFC00115DF000015D839883A0D
:200CA800D0A0091710000326D0A00917103EE83A00000106D0A01104E037883ADFC0011747
:200CB000DF000017DEC00204F800283ADEFFFB04DFC00415DF000315DF000304E13FFE158C
:200CB800E17FFF15E0BFFE171000081601400304E13FFE17000310001007883A00800034A9
:200CC000109825041885883A000001060005883AE0BFFD15E0BFFD1710001026E0BFFD17B9
:200CC800108000171080081710000726E0BFFD171080001710800817E17FFF17E13FFD17C6
:200CD000103EE83A00000A06E0BFFF1700C8000410C001150005883A00000506000329001F
:200CD8001007883A008014441880001500BFFFC4E037883ADFC00117DF000017DEC00204F2
:200CE000F800283ADEFFFE04DFC00115DF000015D839883AD0A0091710000326D0A00917E6
:200CE800103EE83A00000106D0A01104E037883ADFC00117DF000017DEC00204F800283A6C
:200CF000DEFFED04DFC01215DF001115DF001104E13FFF15E0BFFF171000081601400304F8
:200CF800E13FFF17000310001007883A00800034109825041885883A000001060005883A08
:200D0000E0BFEF15E0BFEF1710000E26E0BFEF1710800017108008171000021E0080004458
:200D080000000D06E0BFF004100B883AE13FFF1700032CC0E0BFF1171088002010803FCC29
:200D100000000506000338401007883A00801444188000150005883AE037883ADFC0011788
:200D1800DF000017DEC00204F800283ADEFFFE04DFC00115DF000015D839883AD0A00917DC
:200D200010000326D0A00917103EE83A00000106D0A01104E037883ADFC00117DF00001768
:200D2800DEC00204F800283ADEFFF904DFC00615DF000515DF000504E13FFD15E17FFE1593
:200D3000E1BFFF15E03FFB15E0BFFD171000081601400304E13FFD17000310001007883A77
:200D380000800034109825041885883A000001060005883AE0BFFC15E0BFFC171000102641
:200D4000E0BFFC17108000171080071710000926E0BFFC171080001710800717E1BFFF1790
:200D4800E17FFE17E13FFC17103EE83AE0BFFB150000050600BFDE84E0BFFB1500000206E1
:200D500000BFEBC4E0BFFB15E0BFFB171000070E000346C01007883AE0BFFB170085C83A76
:200D58001880001500BFFFC4E0BFFB15E0BFFB17E037883ADFC00117DF000017DEC00204C2
:200D6000F800283ADEFFFD04DFC00215DF000115DF0001040009883A0003A2C00001883AB9
:200D68000003A6400180003431960804014000342956080401000034211608040004C700B7
:200D7000000482C0010000342112230400054300D0A01217D0E01317D1201417200D883AC8
:200D7800180B883A1009883A00002480E0BFFF150100004400031640E13FFF1700054440E7
:200D8000DEFFFE04DF000115DF000104E13FFF150001883AE037883ADF000017DEC0010432
:200D8800F800283ADEFFFE04DF000115DF000104E13FFF150001883AE037883ADF00001773
:200D9000DEC00104F800283ADEFFFE04DFC00115DF000015D839883AD0A009171000032622
:200D9800D0A00917103EE83A00000106D0A01104E037883ADFC00117DF000017DEC0020485
:200DA000F800283ADEFFF904DFC00615DF000515DF000504E13FFD15E17FFE15E1BFFF150B
:200DA800E0BFFD171000081601400304E13FFD17000310001007883A00800034109825045D
:200DB0001885883A000001060005883AE0BFFB15E0BFFB1710002226E0BFFB1710800217E4
:200DB800108000CC108000601000181EE0BFFB17108000171080051710001426E0BFFB178A
:200DC0001080001710800517E0FFFF17180D883AE17FFE17E13FFB17103EE83AE0BFFC151D
:200DC800E0BFFC171000070E000364801007883AE0BFFC170085C83A1880001500BFFFC40C
:200DD00000000C06E0BFFC1700000A06000364801007883A008003441880001500000406F1
:200DD800000364801007883A008014441880001500BFFFC4E037883ADFC00117DF000017AE
:200DE000DEC00204F800283ADEFFFC04DFC00315DF000215DC000115DF000204E13FFE1561
:200DE800E0BFFE17108000D01000111E0400003484182504E0BFFE17014003041009883AC4
:200DF000000310008085883A10800204100000150400003484182504E0BFFE170140030455
:200DF8001009883A000310008085883A100000150001883AE6FFFF04DFC00217DF000117A7
:200E0000DC000017DEC00304F800283ADEFFF904DF000615DF000604E13FFF150005303A80
:200E0800E0BFFE15E0FFFE1700BFFF841884703A1001703AE0BFFE17E0BFFB15D0A00A17ED
:200E100010C000C400BFFF041884703AD0A00A15D0E00A17E0BFFF171887883A008000B47C
:200E18001080000410C0062EE0BFFB17E0BFFA15E0BFFA171001703A00BFFFC400000B06C5
:200E2000D0A00A17E0BFFD15D0E00A17E0BFFF171885883AD0A00A15E0BFFB17E0BFFC159B
:200E2800E0BFFC171001703AE0BFFD17E037883ADF000017DEC00104F800283ADEFFFE04DF
:200E3000DFC00115DF000015D839883AD0A0091710000326D0A00917103EE83A0000010656
:200E3800D0A01104E037883ADFC00117DF000017DEC00204F800283ADEFFF904DFC00615FD
:200E4000DF000515DF000504E13FFD15E17FFE15E1BFFF15E0BFFD1710000816014003042F
:200E4800E13FFD17000310001007883A00800034109825041885883A000001060005883AB8
:200E5000E0BFFB15E0BFFB1710002126E0BFFB1710800217108000CC10001826E0BFFB1716
:200E5800108000171080061710001426E0BFFB171080001710800617E0FFFF17180D883AFB
:200E6000E17FFE17E13FFB17103EE83AE0BFFC15E0BFFC171000070E00038BC01007883AAD
:200E6800E0BFFC170085C83A1880001500BFFFC400000C06E0BFFC1700000A0600038BC0E0
:200E70001007883A00800344188000150000040600038BC01007883A00801444188000155F
:200E780000BFFFC4E037883ADFC00117DF000017DEC00204F800283ADEFFFD04DFC00215C0
:200E8000DF000115DF000104E13FFF15D1600604E13FFF1700047880E037883ADFC0011748
:200E8800DF000017DEC00204F800283ADEFFFD04DFC00215DF000115DF000104E13FFF15B5
:200E900000051140008000441001703A0001883AE037883ADFC00117DF000017DEC0020480
:200E9800F800283ADEFFFE04DFC00115DF000015D839883A01C0FA04000D883A000B883A2A
:200EA000010000B42104100400045A4001800044000B883A0100003421188F040003C280CE
:200EA800010000342118850400039F800001883AE037883ADFC00117DF000017DEC0020424
:200EB000F800283ADEFFFA04DFC00515DF000415DF000404E13FFD15E17FFE15E1BFFF15FC
:200EB800E0BFFD1710800017E0BFFC15E0BFFC1710C00A04E0BFFD1710800217100F883A43
:200EC000E1BFFF17E17FFE171809883A00040EC0E037883ADFC00117DF000017DEC0020408
:200EC800F800283ADEFFFA04DFC00515DF000415DF000404E13FFD15E17FFE15E1BFFF15E4
:200ED000E0BFFD1710800017E0BFFC15E0BFFC1710C00A04E0BFFD1710800217100F883A2B
:200ED800E1BFFF17E17FFE171809883A00043080E037883ADFC00117DF000017DEC002040E
:200EE000F800283ADEFFFC04DFC00315DF000215DF000204E13FFF15E0BFFF171080001799
:200EE800E0BFFE15E0BFFE1710C00A04E0BFFF1710800217100B883A1809883A0003F9404C
:200EF000E037883ADFC00117DF000017DEC00204F800283ADEFFFA04DFC00515DF000415D2
:200EF800DF000404E13FFD15E17FFE15E1BFFF15E0BFFD1710800017E0BFFC15E0BFFC17DE
:200F000010800A04E1BFFF17E17FFE171009883A0003FFC0E037883ADFC00117DF000017E5
:200F0800DEC00204F800283ADEFFFA04DFC00515DF000415DF000404E13FFD15E17FFE15B3
:200F1000E1BFFF15E0BFFD1700C0004410C00815E0BFFD1710800017108001041007883AA1
:200F1800E0BFFD171080081718800035E0BFFE17E0FFFF17D8000015E1FFFD17018000344B
:200F2000318F3A04180B883A1009883A00048EC0E0BFFD1710000915E0BFFD171080020477
:200F2800D0E01617E1FFFD1701800034318FBD04180B883A1009883A000462001000040E5A
:200F3000E0FFFD1700A0003410BFFFC4188001150001883AE037883ADFC00117DF00001751
:200F3800DEC00204F800283ADEFFF804DF000715DF000704E13FFF15E0BFFF17E0BFFB1545
:200F4000E0BFFB1710800017E0BFFC15E0BFFC171080010410800037E0BFFD15E0BFFD1717
:200F48001080C00C10006D26E0BFFD171080400C1000352600800074E0BFF915E0BFFB173E
:200F500010800A17108000441081FFCCE0BFFE15E0BFFB1710C00B17E0BFFE1718801526C4
:200F5800E0BFFC1710800037E0BFF915E0BFF91710A0000C10001126E0BFFB1710800A173F
:200F6000E0FFF9171809883AE0FFFB171885883A10800E0411000005E0BFFB1710800A1735
:200F68001080004410C1FFCCE0BFFB1710C00A15003FE2060001883A000001060001883AA5
:200F7000E0BFF91710BFFFEC10000F26E0BFFB1710C0081700BFFF841886703AE0BFFB17D8
:200F780010C00815E0BFFC17108001041007883AE0BFFB171080081718800035E0BFFC176D
:200F80001080010410800037E0BFFD171080800C103FBE26E0BFFD171004D43AE0BFFA1570
:200F880000001406E0BFFC17E0FFFB1718C00D17E13FFB1720C7883A18C20E0418C00003EE
:200F900018C03FCC18C0201C18FFE00410C00035E0BFFB1710800D171080004410C1FFCC75
:200F9800E0BFFB1710C00D15E0BFFA1710BFFFC4E0BFFA15E0BFFA1710000526E0BFFB170A
:200FA00010C00D17E0BFFB1710800C1718BFE51EE0BFFA17103F9D26E0BFFB1710C008179D
:200FA80000BFFF441886703AE0BFFB1710C00815E0BFFB1710800017108001041007883A7B
:200FB000E0BFFB171080081718800035E0BFFC171080010410800037003F8C060001883A52
:200FB8000001883AE037883ADF000017DEC00104F800283ADEFFF804DF000715DF000704CC
:200FC000E13FFB15E0BFFB17E0BFF915E0BFF917108000171080010410800037E0BFFA1523
:200FC800E0BFFA171081000C10000B26E0BFF91710800017108001041007883AE0BFF91708
:200FD000108008171081001418800035E0BFF9171000091500000A06E0BFF91710C0091754
:200FD80000A0003410BFFF0410C00536E0BFF9171080091710C00044E0BFF91710C0091538
:200FE000D0A01617E037883ADF000017DEC00104F800283ADEFFFD04DF000215DF000204CF
:200FE800E13FFE15E17FFF1500000506E0BFFF171090000C1000022600BFFD4400000B068D
:200FF000E0BFFE1710C00D17E0BFFE1710800C1718800526E0BFFE1710C00917E0BFFE17B7
:200FF8001080011718BFF1360005883AE037883ADF000017DEC00104F800283ADEFFFA04C5
:20100000DF000515DF000504E13FFD15E17FFE15E1BFFF1500BFF9C4E0BFFB15E0BFFE17B7
:2010080010DA80601800031E109A80A01000181E00002906E0BFFD1710C0011700A0003417
:2010100010BFFFC418802126E0BFFF1710800017E0BFFC15E0BFFC17108000901000061E3D
:20101800E0FFFC1700A0003410BFFFC418800226E0BFFC170000020600A0003410BFFF84C0
:20102000E0FFFD1718800115E03FFB1500000F06E0BFFD1710C0011700A0003410BFFFC4CA
:2010280018800C26E0BFFD1710C00917E0BFFD17108001171885803A10C03FCCE0BFFF17F9
:2010300010C00015E03FFB15000002060001883A000001060001883AE0BFFB17E037883A6D
:20103800DF000017DEC00104F800283ADEFFF304DFC00C15DF000B15DF000B04E13FFC15F3
:20104000E17FFD15E1BFFE15E1FFFF15E0BFFD17E0BFF51500004706E0BFFC1710800A176B
:20104800E0BFF715E0BFFC1710800B17E0BFF815E0FFF717E0BFF81718800536E0FFF71772
:20105000E0BFF8171885C83AE0BFF6150000040600C20004E0BFF8171885C83AE0BFF615C2
:20105800E0BFF61710001E26E0FFFE17E0BFF6171880022EE0BFFE17E0BFF615E0BFFC1700
:2010600010C00E04E0BFF8171885883AE1BFF617100B883AE13FF51700017780E0FFF517E8
:20106800E0BFF6171885883AE0BFF515E0FFFE17E0BFF6171885C83AE0BFFE15E0FFF817D5
:20107000E0BFF6171885883A10C1FFCCE0BFFC1710C00B15E0BFFE1700BFCF1600000106B8
:201078000001883AE0FFF517E0BFFD171880141EE0BFFF171090000C1000131E0001883AC8
:20108000E0BFFC1710C00A17E0BFF7171880051EE0BFFC1710C00917E0BFFC171080011749
:2010880018BFF736E0BFFC1710C00A17E0BFF71718800726E0BFFE1700BFB71600000506E4
:201090000001883A000003060001883A000001060001883AE0FFF517E0BFFD171880182673
:201098000005303AE0BFFB15E0FFFB1700BFFF841884703A1001703AE0BFFB17E0BFFA1587
:2010A000E0BFFC171080081710C00054E0BFFC1710C00815E0BFFC1710800017108001041E
:2010A8001007883AE0BFFC171080081718800035E0BFFA17E0BFF915E0BFF9171001703A5A
:2010B000E0FFF517E0BFFD1718800426E0FFF517E0BFFD171885C83A00000606E0BFFF17C2
:2010B8001090000C1000022600BFFD440000010600BFFEC4E037883ADFC00117DF00001726
:2010C000DEC00204F800283ADEFFF304DFC00C15DF000B15DF000B04E13FFC15E17FFD15EE
:2010C800E1BFFE15E1FFFF15E03FF515E0BFFD17E0BFF71500003706E0BFFC1710800C1738
:2010D000E0BFF915E0BFFC1710800D17E0BFF515E0FFF917E0BFF5171880062EE0FFF517F3
:2010D800E0BFF9171885C83A10BFFFC4E0BFF61500000B06E0BFF5171000052600C20004B1
:2010E000E0BFF9171885C83AE0BFF6150000040600C1FFC4E0BFF9171885C83AE0BFF61572
:2010E800E0BFF61710001E26E0FFFE17E0BFF6171880022EE0BFFE17E0BFF615E0BFFC1770
:2010F00010C20E04E0BFF9171885883AE1BFF617E17FFD171009883A00017780E0FFFD1707
:2010F800E0BFF6171885883AE0BFFD15E0FFFE17E0BFF6171885C83AE0BFFE15E0FFF9173C
:20110000E0BFF6171885883A10C1FFCCE0BFFC1710C00C15E0BFFE1700BFC716000001062E
:201108000001883A0005303AE0BFFB15E0FFFB1700BFFF841884703A1001703AE0BFFB1701
:20111000E0BFFA15E0BFFC171080081710C00094E0BFFC1710C00815E0BFFC171080001754
:20111800108001041007883AE0BFFC171080081718800035E0BFFA17E0BFF815E0BFF81711
:201120001001703AE0BFFE170080100EE0BFFF171090000C1000101E0001883AE0BFFC178E
:2011280010C00D17E0BFF5171880051EE0BFFC1710C00917E0BFFC171080011718BFF7364D
:20113000E0BFFC17108009171000051EE0BFFE1700BFD016000003060001883A00000106DE
:201138000001883AE0FFFD17E0BFF71718800426E0FFFD17E0BFF7171885C83A0000060627
:20114000E0BFFF171090000C1000022600BFFD440000010600BFFEC4E037883ADFC00117DE
:20114800DF000017DEC00204F800283ADEFFFA04DFC00515DF000415DF000404E13FFF15EC
:201150000007883AE0BFFF1710C00035E0BFFF1710800104108000370005303AE0BFFD15CB
:20115800E0FFFD1700BFFF841884703A1001703AE0BFFD17E0BFFC15000500C0E0BFFC1767
:20116000E0BFFE15E0BFFE171001703A0001883AE037883ADFC00117DF000017DEC0020461
:20116800F800283ADEFFF804DFC00715DF000615DF000604E13FFC15E17FFD15E1BFFE1540
:20117000E1FFFF15E0BFFF17E0BFFB15D0A016171000021EE0BFFB17D0A01615E0BFFC173C
:201178001080010400C001C410C00035D8000015E1FFFC170180003431914B04E17FFE171D
:20118000E13FFD1700048EC00001883AE037883ADFC00117DF000017DEC00204F800283A82
:20118800DEFFF504DF000A15DF000A04E13FFC15E17FFD15E1BFFE15E1FFFF15E03FF61512
:20119000D0A0161710003C26E0BFFC1710003826E0BFFC17E0FFFE1710C00315E0BFFC17D0
:20119800E0FFFF1710C005150005303AE0BFF915E0FFF91700BFFF841884703A1001703A0A
:2011A000E0BFF917E0BFF815D0A01717E0BFF615E0FFFD17E0BFF6171885883A10C000447A
:2011A800E0BFFC1710C00215E0BFFC1710C00217E0BFF6171880042EE0BFFC1700C00044C7
:2011B00010C0040500000206E0BFFC1710000405E0BFFC17D0E00C04E0FFFA15E0BFFB1564
:2011B800E0BFFB17E0FFFA1710C00115E0BFFA1710C00017E0BFFB1710C00015E0BFFA17B3
:2011C00010800017E0FFFB1710C00115E0BFFA17E0FFFB1710C00015E0BFF817E0BFF715B2
:2011C800E0BFF7171001703A0005883A0000030600BFFA840000010600BFDE84E037883A91
:2011D000DF000017DEC00104F800283ADEFFFE04DFC00115DF000015D839883AD0A0091721
:2011D80010000326D0A00917103EE83A00000106D0A01104E037883ADFC00117DF000017AC
:2011E000DEC00204F800283ADEFFFA04DFC00515DF000415DF000404E13FFE15E17FFF15D7
:2011E800E0BFFE1710000326E0BFFE17108002171000061E000474C01007883A008005844F
:2011F0001880001500BFFA8400001306E0BFFE17E0FFFF17E0FFFC15E0BFFD15E0BFFD17DF
:2011F800E0FFFC1710C00115E0BFFC1710C00017E0BFFD1710C00015E0BFFC171080001775
:20120000E0FFFD1710C00115E0BFFC17E0FFFD1710C000150005883AE037883ADFC0011714
:20120800DF000017DEC00204F800283ADEFFFD04DFC00215DF000115DF00010400800034B1
:201210001095F004E0BFFF1500000606E0BFFF1710800017103EE83AE0BFFF1710BFFF0413
:20121800E0BFFF15E0FFFF17008000341095F10418BFF62E0001883AE037883ADFC0011772
:20122000DF000017DEC00204F800283ADEFFFD04DFC00215DF000115DF0001040080003499
:201228001095F004E0BFFF1500000606E0BFFF1710800017103EE83AE0BFFF1710BFFF04FB
:20123000E0BFFF15E0FFFF17008000341095F10418BFF62E0001883AE037883ADFC001175A
:20123800DF000017DEC00204F800283ADEFFF904DFC00615DF000515DF000504E13FFC15FC
:20124000E17FFD15E1BFFE15E1FFFF15E0800217D8800015E1FFFF17E1BFFE17E17FFD1770
:20124800E13FFC170004A9C0E037883ADFC00117DF000017DEC00204F800283ADEFFF90488
:20125000DF000615DF000604E13FFE15E17FFF15E0BFFF17E0BFFA150005303AE0BFFB1573
:20125800E0FFFB1700BFFF841884703A1001703AE0BFFB17E0BFFC1500C00044E0BFFA172D
:201260001884983A1007883AD0A015171884B03AD0A01515D0A01517100170FAE0BFFC17A2
:20126800E0BFFD15E0BFFD171001703A0005883A0001883AE037883ADF000017DEC001044B
:20127000F800283ADEFFF904DF000615DF000604E13FFE15E17FFF15E0BFFF17E0BFFA153D
:201278000005303AE0BFFB15E0FFFB1700BFFF841884703A1001703AE0BFFB17E0BFFC15A3
:2012800000C00044E0BFFA171884983A0084303A1007883AD0A015171884703AD0A01515E9
:20128800D0A01517100170FAE0BFFC17E0BFFD15E0BFFD171001703A0005883A0001883AD4
:20129000E037883ADF000017DEC00104F800283ADEFFFC04DF000315DF000304E13FFE1585
:20129800E17FFF15000530FAE0BFFD1500C00044E0BFFF171884983A1007883AE0BFFD172F
:2012A0001884703A1004C03A10803FCCE037883ADF000017DEC00104F800283ADEFFF5049D
:2012A800DFC00A15DF000915DF000904E13FFC15E17FFD15E1BFFE15E1FFFF1500BFFA84F8
:2012B000E0BFF715E0BFFD17E0BFF815E0BFF817108008081000271E0005303AE0BFFB1553
:2012B800E0FFFB1700BFFF841884703A1001703AE0BFFB17E0BFFA1500800034109CC0045F
:2012C000E0FFF817180690FA10C5883AE0FFFE1710C0001500800034109CC004E0FFF817F6
:2012C800180690FA10C5883A10800104E0FFFF1710C00015E0BFFE1710000526E0BFF817BB
:2012D000100B883AE13FFC17000493C000000406E0BFF817100B883AE13FFC1700049C40EF
:2012D800E0BFF715E0BFFA17E0BFF915E0BFF9171001703AE0BFF717E037883ADFC0011747
:2012E000DF000017DEC00204F800283ADEFFF804DFC00715DF000615DC000515DF0006048D
:2012E800E13FFB15E17FFC15E1BFFD15E1FFFE15E1BFFE17E17FFD17E13FFC170004E1401F
:2012F000E0BFFA15E0BFFA17100022160400003484182504E0BFFA17014003041009883A68
:2012F800000310008085883A10C00017E0BFFB1710C000150400003484182504E0BFFA17D2
:20130000014003041009883A000310008085883A1080010410C00017E0BFFB1710C00115BD
:201308000400003484182504E0BFFA17014003041009883A000310008085883A1080020485
:2013100010C00017E0BFFB1710C00215E13FFA17000378800001883AE6FFFF04DFC00217AF
:20131800DF000117DC000017DEC00304F800283ADEFFFB04DFC00415DF000315DF0003045B
:20132000E13FFD15E17FFE15E1BFFF1501C07FC401800044E17FFD1701000034211828047D
:201328000004B8C001C07FC4000D883AE17FFE1701000034211825040004B8C001C07FC4CA
:2013300001800044E17FFF170100003421182B040004B8C00001883AE037883ADFC00117F6
:20133800DF000017DEC00204F800283ADEFFFE04DFC00115DF000015D839883AD0A00917B6
:2013400010000326D0A00917103EE83A00000106D0A01104E037883ADFC00117DF00001742
:20134800DEC00204F800283ADEFFFB04DFC00415DF000315DC000215DF000304E13FFE15F0
:20135000E0BFFE171080021710D00034E0BFFE1710C00215E03FFD150000230604000034DF
:2013580084182504E0BFFD17014003041009883A000310008085883A10C00017E0BFFE1765
:20136000108000171880151E0400003484182504E0BFFD17014003041009883A0003100015
:201368008085883A108002041080001710000B0E01400304E13FFD17000310001007883AD0
:2013700000800034109825041887883AE0BFFE171880022600BFFCC400000806E0BFFD17C3
:2013780010800044E0BFFD15D0A008171007883AE0BFFD1718BFD92E0005883AE6FFFF0428
:20138000DFC00217DF000117DC000017DEC00304F800283ADEFFF604DFC00915DF0008151C
:20138800DF000804E13FFD15E17FFE15E1BFFF1500BFFFC4E0BFF91500BFFB44E0BFFA1526
:20139000E03FFB15D1600604E13FFD1700051380E0BFF815E0BFF8171000051EE13FFD1746
:2013980000051C80E0BFF81500800044E0BFFB15E0BFF81710002B26E13FF81700052D0005
:2013A000E0BFF915E0BFF9171000030EE0BFF917E0BFFA150000250601400304E13FF917B0
:2013A800000310001007883A00800034109825041885883AE0BFFC15E0FFFE1700900034ED
:2013B00010BFFFC41886703AE0BFFC1710C00215E0BFFB171000051EE13FFC170004D2803D
:2013B800E0BFFA15E0BFFA1710001016E0BFF8171080031710000826E0BFF8171080031793
:2013C000E1FFFF17E1BFFE17E17FFD17E13FFC17103EE83A000001060005883AE0BFFA15CF
:2013C8000000020600BFFB44E0BFFA15E0BFFA171000090EE13FF917000378800004CEC0BD
:2013D0001007883AE0BFFA170085C83A1880001500BFFFC400000106E0BFF917E037883A2F
:2013D800DFC00117DF000017DEC00204F800283ADEFFFA04DF000515DF000504E13FFF155A
:2013E0000005303AE0BFFC15E0FFFC1700BFFF841884703A1001703AE0BFFC17E0BFFB1538
:2013E800E0BFFF17E0BFFD15E0BFFD1710800017E0FFFD1718C0011710C00115E0BFFD17A9
:2013F00010800117E0FFFD1718C0001710C00015E0BFFD17E0FFFD1710C00115E0BFFD172F
:2013F800E0FFFD1710C00015E0BFFB17E0BFFE15E0BFFE171001703A0001883AE037883A8F
:20140000DF000017DEC00104F800283ADEFFFB04DFC00415DF000315DF000304D0A00C17D5
:20140800E0BFFD15D0A0171710800044D0A0171500002E06E0BFFD1710800017E0BFFE15C5
:20141000E0BFFD171080040310803FCC10000426D0A017171000021EE0BFFD171000040503
:20141800E0BFFD1710800217D0E0171718801D36E0BFFD171080040310803FCC1000191E63
:20142000E0BFFD1710800317E0FFFD1718C005171809883A103EE83AE0BFFF15E0BFFF17AD
:201428001000031EE13FFD170004F70000000D06E0BFFD1710C00217E0BFFF171887883A7F
:20143000E0BFFD1710C00215E0BFFD1710C00217D0A017171880032EE0BFFD1700C0004448
:2014380010C00405E0BFFE17E0BFFD15E0FFFD17D0A00C0418BFCF1E0001883A0001883A99
:20144000E037883ADFC00117DF000017DEC00204F800283ADEFFFF04DF000015D839883A61
:20144800000170FA0001883AE037883ADF000017DEC00104F800283ADEFFFA04DFC00515F6
:20145000DF000415DF000404E13FFE15E17FFF15E0BFFF1710800017E0BFFC15E13FFE17B5
:2014580000003F0010800044E0BFFD1500000D06E0BFFC1710800217E0FFFD17180D883A68
:20146000E17FFE171009883A000547C01000021EE0BFFC1700000706E0BFFC1710800017C8
:20146800E0BFFC15E0FFFC17E0BFFF1718BFF01E0005883AE037883ADFC00117DF000017DB
:20147000DEC00204F800283ADEFFFB04DFC00415DF000315DF000304E13FFF15D0A004172E
:20147800E0BFFD1500003106E0BFFD17108002171009883A00003F00E0BFFE15E0BFFD1791
:2014800010C00217E0BFFE1710BFFFC41885883A1080000310803FCC1080201C10BFE00411
:2014880010800BD81000031EE0BFFE1710BFFFC4E0BFFE15E0BFFE17E0FFFF171885883AA0
:201490001080000310803FCC1080201C10BFE00410800BE01000081EE0BFFE17E0FFFF1735
:201498001885883A1080000310803FCC1080201C10BFE00410000A1EE0BFFD171080021794
:2014A000E0FFFE17180D883AE17FFF171009883A000547C01000021EE0BFFD170000070604
:2014A800E0BFFD1710800017E0BFFD15E0FFFD17D0A0040418BFCC1E0005883AE037883A4D
:2014B000DFC00117DF000017DEC00204F800283ADEFFFA04DFC00515DF000415DC000315F1
:2014B800DF000404E13FFE1500BFFA04E0BFFD15E03FFC1500001D0604000034841825043C
:2014C000E0BFFC17014003041009883A000310008085883A108000171000111E040000343F
:2014C80084182504E0BFFC17014003041009883A000310008085883AE0FFFE1710C00015B7
:2014D000D0E00817E0BFFC171880020EE0BFFC17D0A00815E0BFFC17E0BFFD150000060625
:2014D800E0BFFC1710800044E0BFFC15E0BFFC1710800810103FE01EE0BFFD17E6FFFF047C
:2014E000DFC00217DF000117DC000017DEC00304F800283ADEFFFE04DF000115DF00010493
:2014E800E13FFF15E0BFFF1710BFFE8410C0042818001A1E100690BA008000341094F304AF
:2014F0001885883A108000171000683A0000540C0000540C0000541C0000541C0000541C14
:2014F8000000540C000054140000541C0000540C0000540C0000541C0000540C00005414A4
:201500000000541C0000541C0000540C00800044000003060005883A000001060005883A29
:20150800E037883ADF000017DEC00104F800283A200B883A000F883A000D883A0009883A9F
:2015100000054F81DEFFFE04000B883ADC000015DFC001152021883A000561000080003477
:20151800109C9D041100001720800F1710000126103EE83A8009883A0005790001C000C483
:201520003980192E2144B03A11C4703A10000F262080000328C0000310C0151E31BFFF8494
:2015280001FFFFC4000004062080000328C0000331BFFFC410C00E1E210000442940004487
:2015300031FFF91E0005883AF800283A20C000172880001718BFEE1E31BFFF042100010481
:201538002940010439BFF936303FE91E003FF50610C5C83AF800283ADEFFFA04DC0003154E
:2015400004000034841C9D0480C00017DC400415DFC00515188052172023883A100037265A
:2015480010C00117010007C420C00E161A0000448800221E18C0008418C7883A18C7883A07
:201550001200011510C7883A194000150005883ADFC00517DC400417DC000317DEC00604F5
:20155800F800283A00800034108000041000262601006404D9400015D9800115D9C00215BF
:2015600000000000D9400017D9800117D9C0021710001D26810000171000011502000044C1
:20156800224052170007883A12400015208052151000621510006315883FDE2618C9883AE4
:201570002109883A1109883A21802215018000441240621730CC983A4992B03A12406215CF
:2015780021C0421501000084893FD21E11006317218CB03A11806315003FCE0618805304B1
:2015800018805215003FC60600BFFFC4003FD006DEFFF504DF000915DD400615DC8003152B
:20158800DFC00A15DDC00815DD800715DD000515DCC00415DC400215DC000115D900001593
:201590002839883A04800044057FFFC400800034109C9D04120000174500521744C05204D7
:20159800A0001C26A080011715FFFFC4B8000D16140000448421883A8421883A8440200459
:2015A000A463883AA421883AE0001E2680804017E0801C26BDFFFFC4843FFF048C7FFF046B
:2015A800BD7FF91E008000341080000410000926A08001171000301EA08000171000322614
:2015B000A009883A98800015000000009D000017A03FE41EDFC00A17DF000917DDC0081773
:2015B800DD800717DD400617DD000517DCC00417DC800317DC400217DC000117DEC00B0462
:2015C000F800283AA080011780C0001710BFFFC415C0142680000015183FDE2695C8983A62
:2015C800A0806217A58001172084703A10000B26A08063172088703A20000C1E8940001788
:2015D000D9000017183EE83AA080011715BFBF1E98800017153FCF26003FBC06183EE83AB9
:2015D800003FF906A5C00115003FEB0689000017183EE83A003FF406A0800017A027883AF9
:2015E0001029883A003FB6060005883A003FFB06DEFFFD04DF000215DF000204E13FFF1501
:2015E8000001883AE0BFFF17E0BFFE15E0BFFE1710000226002AF07000000106002AF0B072
:2015F000003FFF060000001000000010000000050000001000000010000000200000001022
:2015F80000000010000000F1000000F1000000F100000011000000D1000000F1000000F12C
:201600000000001164616552000000790000000A000000437665642F6C756E2F0000006C1F
:201608007665642F61746A2F61755F67000074727665642F61746A2F61755F670000747206
:201610000000000000005B2C00005B9400005BFC00000000000000000000000000000000ED
:2016180000000000000000000000000000000000000000000000581000000000000000004A
:201620000000000000000000000000000000000000000000000000000000000000000000AA
:201628000000000000000000000000000000000000000000000000000000000000000000A2
:2016300000000000000000000000000000000000000000000000000000000000000000009A
:20163800000000000000000100000000ABCD330EE66D12340005DEEC0000000B0000000065
:2016400000000000000000000000000000000000000000000000000000000000000000008A
:20164800000000000000000000000000000000000000000000000000000000000000000082
:2016500000000000000000000000000000000000000000000000000000000000000000007A
:20165800000000000000000000000000000000000000000000000000000000000000000072
:2016600000000000000000000000000000000000000000000000000000000000000000006A
:20166800000000000000000000000000000000000000000000000000000000000000000062
:2016700000000000000000000000000000000000000000000000000000000000000000005A
:20167800000000000000000000000000000000000000000000000000000000000000000052
:2016800000000000000000000000000000000000000000000000000000000000000000004A
:20168800000000000000000000000000000000000000000000000000000000000000000042
:2016900000000000000000000000000000000000000000000000000000000000000000003A
:20169800000000000000000000000000000000000000000000000000000000000000000032
:2016A00000000000000000000000000000000000000000000000000000000000000000002A
:2016A800000000000000000000000000000000000000000000000000000000000000000022
:2016B00000000000000000000000000000000000000000000000000000000000000000001A
:2016B800000000000000000000000000000000000000000000000000000000000000000012
:2016C00000000000000000000000000000000000000000000000000000000000000000000A
:2016C800000000000000000000000000000000000000000000000000000000000000000002
:2016D0000000000000000000000000000000000000000000000000000000000000000000FA
:2016D8000000000000000000000000000000000000000000000000000000000000000000F2
:2016E0000000000000000000000000000000000000000000000000000000000000000000EA
:2016E8000000000000000000000000000000000000000000000000000000000000000000E2
:2016F0000000000000000000000000000000000000000000000000000000000000000000DA
:2016F8000000000000000000000000000000000000000000000000000000000000000000D2
:201700000000000000000000000000000000000000000000000000000000000000000000C9
:201708000000000000000000000000000000000000000000000000000000000000000000C1
:201710000000000000000000000000000000000000000000000000000000000000000000B9
:2017180000000000000000000000000000005C6400005C6400005C6C00005C6C00005C74D1
:2017200000005C7400005C7C00005C7C00005C8400005C8400005C8C00005C8C00005C94A9
:2017280000005C9400005C9C00005C9C00005CA400005CA400005CAC00005CAC00005CB4A1
:2017300000005CB400005CBC00005CBC00005CC400005CC400005CCC00005CCC00005CD499
:2017380000005CD400005CDC00005CDC00005CE400005CE400005CEC00005CEC00005CF491
:2017400000005CF400005CFC00005CFC00005D0400005D0400005D0C00005D0C00005D1484
:2017480000005D1400005D1C00005D1C00005D2400005D2400005D2C00005D2C00005D3479
:2017500000005D3400005D3C00005D3C00005D4400005D4400005D4C00005D4C00005D5471
:2017580000005D5400005D5C00005D5C00005D6400005D6400005D6C00005D6C00005D7469
:2017600000005D7400005D7C00005D7C00005D8400005D8400005D8C00005D8C00005D9461
:2017680000005D9400005D9C00005D9C00005DA400005DA400005DAC00005DAC00005DB459
:2017700000005DB400005DBC00005DBC00005DC400005DC400005DCC00005DCC00005DD451
:2017780000005DD400005DDC00005DDC00005DE400005DE400005DEC00005DEC00005DF449
:2017800000005DF400005DFC00005DFC00005E0400005E0400005E0C00005E0C00005E143C
:2017880000005E1400005E1C00005E1C00005E2400005E2400005E2C00005E2C00005E3431
:2017900000005E3400005E3C00005E3C00005E4400005E4400005E4C00005E4C00005E5429
:2017980000005E5400005E5C00005E5C00005E6400005E6400005E6C00005E6C00005E7421
:2017A00000005E7400005E7C00005E7C00005E8400005E8400005E8C00005E8C00005E9419
:2017A80000005E9400005E9C00005E9C00005EA400005EA400005EAC00005EAC00005EB411
:2017B00000005EB400005EBC00005EBC00005EC400005EC400005ECC00005ECC00005ED409
:2017B80000005ED400005EDC00005EDC00005EE400005EE400005EEC00005EEC00005EF401
:2017C00000005EF400005EFC00005EFC00005F0400005F0400005F0C00005F0C00005F14F4
:2017C80000005F1400005F1C00005F1C00005F2400005F2400005F2C00005F2C00005F34E9
:2017D00000005F3400005F3C00005F3C00005F4400005F4400005F4C00005F4C00005F54E1
:2017D80000005F5400005F5C00005F5C00005F6400005F6400005F6C00005F6C00005F74D9
:2017E00000005F7400005F7C00005F7C00005F8400005F8400005F8C00005F8C00005F94D1
:2017E80000005F9400005F9C00005F9C00005FA400005FA400005FAC00005FAC00005FB4C9
:2017F00000005FB400005FBC00005FBC00005FC400005FC400005FCC00005FCC00005FD4C1
:2017F80000005FD400005FDC00005FDC00005FE400005FE400005FEC00005FEC00005FF4B9
:2018000000005FF400005FFC00005FFC00006004000060040000600C0000600C00006014AB
:20180800000060140000601C0000601C00006024000060240000602C0000602C00006034A0
:20181000000060340000603C0000603C00006044000060440000604C0000604C0000605498
:20181800000060540000605C0000605C0000728C0000728C0000581400000000000000001C
:2018200000000000000032640000000000000000000000000000606C000000000000000046
:201828000000606C00000000000000000000606C0000000000000000000000000000000008
:20183000000000000000000000000000000000000000000000000000000000000000000098
:20183800000000000000000000000000000000000000000000000000000000000000000090
:20184000000000000000000000000000000000000000000000000000000000000000000088
:20184800000000000000000000000000000000000000000000000000000000000000000080
:20185000000000000000000000000000000000000000000000000000000000000000000078
:20185800000000000000000000000000000000000000000000000000000000000000000070
:20186000000000000000000000000000000000000000000000000000000000000000000068
:20186800000000000000000000000000000000000000000000000000000000000000000060
:20187000000000000000000000000000000000000000000000000000000000000000000058
:20187800000000000000000000000000000000000000000000000000000000000000000050
:201880000000000000000000000000000000000000000000000000000000000000005830C0
:201888000000000000003B8400003AC400003B24000000000000000000003BD4000210689B
:201890000000000A000000000000000000000000000000000000000000000000000000002E
:20189800000000000000000000000000000000000000000000000000000000000000000030
:2018A000000000000000000000000000000000000000000000000000000000000000000028
:2018A800000000000000000000000000000000000000000000000000000000000000000020
:2018B000000000000000000000000000000000000000000000000000000000000000000018
:201C980000000000000000000000000000000000000000000000584000005840FFFFFFFF00
:201CA0000002000000007284000072840000606C0000606CFFFFFFFF00000000000074002E
:201CA800FFFFFFFF000072A4000072A40000000000000000000000000000000000000000F4
:201CB000000000000000000000000000000000000000000000000000000000000000000014
:201CB80000000000000000000000000000000000000000000000000000000000000000000C
:201CC000000000000000000000000000000000000000000000000000000000000000000004
:201CC8000000000000000000000000000000000000000000000000000000000000000000FC
:00000001FF
